:10488E000000090101240200000301FA0400FA05E8
:10489E0000020A0A5A0B000F0C00FA0D00030E005C
:1048AE00030F0132100096120132130AFA1401029C
:1048BE0015000017010A18010A1905321A010A1B00
:1048CE00010A1C053223011E2400642A00FA2B0063
:1048DE00FA2C50782D003C2E00462F001E3000641E
:1048EE003250783301013432FA35016436016437BF
:1048FE000150380A643C00643E003C3F0001400019
:10490E002D411450420A5A430AC8440532450078D4
:10491E004600FA4701234803034C00FA4EFFFF50AE
:10492E000202510596521432530B28540A9656021F
:10493E0003570546590A465A32FA5B010A5C14328D
:10494E005E000A5F00FE61FFFF6402126701036AE8
:10495E000A3C6B00006C3296780132790132FAFA19
:10496E00FA0065006F00790083008D009700A100AA
:10497E00AC00B600C000CA00D400DE00E800F200B1
:10498E005B0063006A0072007A0082008900910069
:10499E009900A100A800B000B800BF00C700CF006A
:1049AE00D600DF00E600EE00F600400046004C00A8
:1049BE00520059005F0065006B00710077007D00AA
:1049CE00830089008F0095009C00A200A800AE0015
:1049DE00B400BA00C000C600CC00D200D900DF007F
:0549EE00E500EB00F103
:10009E00AE32AF33740A8E048F05FF1200858C3496
:1000AE008D35AE32AF33740A8E048F05FF124B0CB2
:1000BE008C328D33E53345326013740AC39533FFAA
:1000CE00E49532FE8E328F337834124B58E54FA8BA
:1000DE0034B80015D395354010E54FC39535FFE480
:1000EE009534FE8E348F358010E54F2424C395351C
:1000FE00FFE49534FE8E348F35AE34AF3574246FF5
:10010E004E700B753523753400754F018003754F96
:10011E000022900083E0B40104C20B8002D20B9047
:10012E0000C1E075F0DCA4FFAEF0740A8E048F05FA
:10013E00FF1200859007A9ECF0A3EDF0A20840167F
:10014E0074038C068D07124AF17401124AE390076C
:10015E00A7EEF0A3EFF07E017F0090007FE0124A41
:10016E00F19000C2E08E048F05FF120085740AFF25
:10017E001200858D389000CBE075F0DCA4FFAEF058
:10018E00740A8E048F05FF1200859007ADECF0A364
:10019E00EDF09000C7E0B402089000A9E0640260A0
:1001AE0002800674019000A9F09000ACE0B40B0838
:1001BE0074E390006EF080499000ACE0B419129098
:1001CE0000C2E090495A124AD4E49390006EF08037
:1001DE00309000ACE0B41E129000C2E0904978124C
:1001EE004AD4E49390006EF080179000ACE0B428EF
:1001FE00109000C2E09049A2124AD4E49390006E8F
:10020E00F09000DFE0B4011790002A740FF0A37491
:10021E00FFF090002CE4F0A3F074029000DFF09059
:10022E0000DFE0B4034190002CE0FEA3E0FF90005D
:10023E002AE0FCA3E0FD124B507410124AF1740830
:10024E00124AE3EF90006BF0EF700674FF90006BB4
:10025E00F074009000DFF090002BE090006CF090B6
:10026E00002AE090006DF0900070E0900036F09063
:10027E000036E0D39412400D900036E0C3941290F5
:10028E000037F0800A900036E02412900037F0908C
:10029E000036E0B4240E9000367401F090003A74EB
:1002AE0001F0800590003AE4F0900037E0B4240E9F
:1002BE009000377401F090003B7401F080059000BF
:1002CE003BE4F0900070E0FE9000D3E02E90003DF5
:1002DE00F090003DE0D39424400B90003DE0C39499
:1002EE002490003DF090003DE0B41206741390008F
:1002FE003DF090003DE0B4240690003D7401F09076
:10030E00003DE0D39412400D90003DE0C394129056
:10031E00003EF0800A90003DE0241290003EF090E6
:10032E0000B6E0900038F0900038E0B41206741376
:10033E00900038F0900038E0D39412400D900038C1
:10034E00E0C39412900039F0800A900038E0241235
:10035E00900039F022C293C294C291C292C287C257
:10036E0090E5B554EFF5B5E5B554DFF5B5C296C2D7
:10037E0095C2A0C297C2A2C2A1E5B5547FF5B5E55C
:10038E00B554BFF5B5E5B554FBF5B5C20D7536469A
:10039E009000B9E07005754802800375480390001F
:1003AE001274FFF0A374DCF090009AE0900018F83D
:1003BE00E4F0E8A3F0C212C21474C890002EF074D8
:1003CE00C8900032F0752500752400C208756B00C8
:1003DE00E54AB40903754A00753B00900020E4F02D
:1003EE00A3F0754B1E752700752600C210C2119022
:1003FE0007A9E0FEA3E0FF7403124AF17401124A4A
:10040E00E39007A7EEF0A3EFF0C203900016E4F01E
:10041E00A3F0C21A90001074FFF0A374DCF09000E9
:10042E000C74FFF0A374DCF090000E74FFF0A37454
:10043E00DCF090000474FFF0A374DCF090000674FE
:10044E00FFF0A374DCF022053C2285A74E75A710A1
:10045E009000D5E0C394025014A2D8B34004C293C6
:10046E00C294A2D9B34004C291C292801CA2D8B346
:10047E004002C293A2D9B34002C291A2DAB34002A3
:10048E00C294A2DBB34002C29275D840854EA72219
:10049E00900047E4936406600280FE74C89007AF34
:1004AE00F8E4F0E8A3F075B50075840175A7007542
:1004BE00FF8075EF0690003CE4F075C91075A70F2C
:1004CE0075A1C775A70075D90075CE0C75A70F75E8
:1004DE00F1FE75F2FF75F30775F47875A4BA75A57C
:1004EE00FF75A60775AE0075AFFF75D48175D5FF84
:1004FE0075D6FF75D7FF75A70075A20175A1477553
:10050E00F80975D80075D90475A71075D80075D976
:10051E000475DA0975DB0975DC0975DD0975D840D6
:10052E0075A70075E60075E71075BC0175BE0475FC
:10053E00BD6C75BE0775BDA075BE0875BD0175BCD9
:10054E000075BB1875BC2075BA0875E88075D11397
:10055E0075A70F75E10575E20075C740C293C29489
:10056E00C291C292C287C290E5B554EFF5B5E5B51A
:10057E0054DFF5B5C296C295C2A0C297C2A2C2A15F
:10058E00E5B5547FF5B5E5B554BFF5B5E5B554FB06
:10059E00F5B5759700759780740A1200757597C03A
:1005AE00E5975420700280F8758F0275A700D2AFC0
:1005BE0075980075A90C75A70F75AB4375ADFB75D6
:1005CE00AC1E75A71075C91875CA0075CB0075C815
:1005DE000475A700758912758E04758C00758A00D6
:1005EE00C2A9D28C758D00758B00D2ABD28E75D907
:1005FE0044753100753000752D00752C0075450061
:10060E00754600C2997509C8750800122B7A75B522
:10061E000074639007AFF8E4F0E8A3F0122E0675AD
:10062E000964750800122B7AC219900059E0B401C2
:10063E0008A2B54002D219802E900059E0B40211E2
:10064E0075A70F75F30F75A700A2A34002D21980EC
:10065E0016900059E0B4030F75A70F75F31775A721
:10066E0000A2A44002D219A219B3500302075C746F
:10067E00089007AFF8E4F0E8A3F0122CD5750964E2
:10068E00750800122B7A74099007AFF8E4F0E8A30E
:10069E00F0122CD5750964750800122B7A740A9025
:1006AE0007AFF8E4F0E8A3F0122CD57509647508CD
:1006BE0000122B7A740B9007AFF8E4F0E8A3F01257
:1006CE002CD5750964750800122B7A740C9007AF3F
:1006DE00F8E4F0E8A3F0122CD57509647508001241
:1006EE002B7A740D9007AFF8E4F0E8A3F0122CD536
:1006FE00750964750800122B7A740E9007AFF8E432
:10070E00F0E8A3F0122CD5750964750800122B7A47
:10071E0074029000B8F0900059E090007CF09000C8
:10072E0059E0B401087400900084F0801C900059C8
:10073E00E0B4020874009000C7F0800D900059E0FC
:10074E00B4030674009000D4F0D217020835900757
:10075E00AFE4F0A304F0122CD575096475080012ED
:10076E002B7A74029007AFF8E4F0E8A3F0122CD5C0
:10077E00750964750800122B7A74039007AFF8E4BC
:10078E00F0E8A3F0122CD5750964750800122B7AC7
:10079E0074049007AFF8E4F0E8A3F0122CD57509B5
:1007AE0064750800122B7A74059007AFF8E4F0E830
:1007BE00A3F0122CD5750964750800122B7A7406F5
:1007CE009007AFF8E4F0E8A3F0122CD57509647524
:1007DE000800122B7A74079007AFF8E4F0E8A3F044
:1007EE00122CD5750964750800122B7A74019000CD
:1007FE00B8F0900059E090007CF0900059E0B40100
:10080E00087400900084F0801C900059E0B4020837
:10081E0074009000C7F0800D900059E0B403067488
:10082E00009000D4F0C217122F7A9000C2E070062A
:10083E00740A9000C2F090006EE0700674E39000AF
:10084E006EF0120120E5B54401F5B574069000482E
:10085E00F07401900049F0740390004BF074049012
:10086E00004CF0743490004DF0740590004EF0740E
:10087E000390004FF07400900054F07400900055F7
:10088E00F07401900056F07400900057F074FF90D1
:10089E000058F07452900146F07458900147F0746D
:1008AE0038900148F07420900149F0743390014A59
:1008BE00F0743690014BF0742D90014CF074319021
:1008CE00014DF0742090014EF0743290014FF0748F
:1008DE0052900150F0746F900151F0747490015267
:1008EE00F0746F900153F07472900154F09000DE2A
:1008FE00E090006BF0900095E090006CF090009608
:10090E00E090006DF0C212C21474C890002EF07404
:10091E00C8900032F090001074FFF0A374DCF090D9
:10092E00000C74FFF0A374DCF090000E74FFF0A3C3
:10093E0074DCF090000474FFF0A374DCF0900006F9
:10094E0074FFF0A374DCF0C210C211A2B6B3920908
:10095E00A2B3B3920A752500752400753646754B01
:10096E001E900067E4F075261975276490001274C6
:10097E00FFF0A374DCF0C20D754A00C208752900A1
:10098E00752800900016E4F0A3F0743A90076FF00B
:10099E0074FD900770F0756C00900068E4F0752B94
:1009AE0000752A0090001AE4F0A3F090009AE090EF
:1009BE000018F8E4F0E8A3F090007BE075F032A4A4
:1009CE00FFAEF0900028EEF0A3EFF09007A9E0FE46
:1009DE00A3E0FF7403124AF17401124AE39007A7D1
:1009EE00EEF0A3EFF075490174FA900044F0C21ACC
:1009FE00756B00753B00C20EC20FC21BC203754C55
:100A0E0000C204D205C206D207D21874FE90003F6F
:100A1E00F074FE900040F075370075430075390094
:100A2E00753D32753E00753F00743C900042F07487
:100A3E003C900043F07540007541007542009000F7
:100A4E0020E4F0A3F0754400D2B2D2A4D2B0D2B159
:100A5E00D2A3D2A7D2A6D2A5D2B790007BE0D394D0
:100A6E00FA400674FA90007BF07E017F0090006DD4
:100A7E00E0124AF190006CE02FFF50010E90002A18
:100A8E00EEF0A3EFF0EFD394FFEE940F400790003B
:100A9E002AE4F0A3F090006BE0700674FF90006BF8
:100AAE00F09000B8E0D39402400674019000B8F0C4
:100ABE009000B9E0700575480280037548039000F8
:100ACE00BAE0D39401400674009000BAF09000C0D2
:100ADE00E0C3940A5006740A9000C0F09000CAE079
:100AEE00700674019000CAF09000CAE0B4FF06745C
:100AFE00FE9000CAF09000D1E0D394FE400674FE42
:100B0E009000D1F074019000D7F074019000D8F0ED
:100B1E0074009000DAF074009000DFF0D29CD2ECFA
:100B2E0075CF01A298B35003020F0CC298E546642C
:100B3E00046006E59964FF6002801EE54660087455
:100B4E00E62546900044F0754600E545600874F0D1
:100B5E002545900044F0754500E5466003020C09FA
:100B6E00754600E599B4FF03754501E599B4FE039A
:100B7E00754502E599B4FD03754503E599B4FC038B
:100B8E00754504E599B4FA03754505E599B4FB037B
:100B9E00754601E599B4F903754604E599D394E5D4
:100BAE004007E599C394F040028016859947754633
:100BBE00027E017F00E547C394E6124AF18E2E8F26
:100BCE002F753100753000E599D394C74007E5992C
:100BDE00C394E64002801F85994775460374E5C3AA
:100BEE009547F52F752E00AE2EAF2F90472412008D
:100BFE00647830124B36D299020F0CE546B40102DE
:100C0E008003020CE5E53145307003120363AE300C
:100C1E00AF3190006F124B18E599F07830124B58A7
:100C2E00AE30AF31EFB40106EEB407028003020C12
:100C3E00E590076FE0B43C028003020CCFC29C1219
:100C4E00012090006BE09000DEF090006CE09000D0
:100C5E0095F090006DE0900096F0A2174031754F20
:100C6E0001E54FD394075025E54F9007AFF8E4F018
:100C7E00E8A3F074AA90003CF0122BA675096475D7
:100C8E000800122B7A784F740126F650D4802F75F7
:100C9E004F08E54FD3940E5025E54F9007AFF8E47B
:100CAE00F0E8A3F074AA90003CF0122BA67509642C
:100CBE00750800122B7A784F740126F650D4122F35
:100CCE007A74C89007AFF8E4F0E8A3F0D29C7546AA
:100CDE00007545007599FBE546B4027DE53145305A
:100CEE00700685992D752C00AE30AF3174016F4EA4
:100CFE00701BAC2CAD2DAA2EAB2FED2BFBEC3AFAC4
:100D0E008A068B0790006F124B18E599F078301217
:100D1E004B58AE30AF3174026F4E703DAC2CAD2DD2
:100D2E00740D6D4C702774639007AFF8E4F0E8A370
:100D3E00F074AB90003CF090007CE0900059F01203
:100D4E002EDF74C89007AFF8E4F0E8A3F01201208C
:100D5E00854799754600754500E546B4033FAE30AC
:100D6E00AF3190006F124B18E599F07830124B5856
:100D7E00AE30AF31AC2EAD2F8F028E038C068D07A9
:100D8E00904760120064E493F9740193FEEAD39ED7
:100D9E00EB994009854799754600754500E546B4BF
:100DAE0004028003020F0CE5314530700312036319
:100DBE00AE30AF3190006F124B18E599F0783012CB
:100DCE004B58AE30AF31EFB40006EEB401028003E3
:100DDE00020F0C900052E075F002A4FDACF08D4FA6
:100DEE00ED90006F124B2DEDFAE0FBEA90007212BF
:100DFE004B2DEBFAE0FBEA2BFA900052E0B5020223
:100E0E008003020EFE0DED90006F124B2DE54FFD8F
:100E1E00E0FAED900073124B2DEAFDE0FAEDC39A65
:100E2E00FD900052E0B505028003020EFEE54F90E4
:100E3E000071124B2DE54FFDE0FAED900074124B50
:100E4E002DEAFDE0FAED2AFD900052E0B505028094
:100E5E0003020EFEE54F900075124B2DFDE0FAEDEC
:100E6E00900052E0F4042A900059F0E54F9000767D
:100E7E00124B2DFDE0FAED900052E0F4042A9000A2
:100E8E005AF0E54F900077124B2DFDE0FAED9000F1
:100E9E0052E0F4042A90005BF0E54F900078124B7C
:100EAE002DFDE0FAED900052E0F4042A9007AFF821
:100EBE00E4F0E8A3F074AB90003CF0122EDF75095D
:100ECE0064750800122B7A9007AF124AFF122EDFBC
:100EDE00750964750800122B7A9007AF124AFF123B
:100EEE002EDF7599F9750964750800122B7A80FE4C
:100EFE007599FF750964750800122B7A80FEE54519
:100F0E006006A299B3B3400302106DC299E545B4D1
:100F1E00011FAE30AF31900048124B18E0F59978B2
:100F2E0030124B58AE30AF3174116F4E70037545A1
:100F3E0000E545B40203854999E545B4031DAE307D
:100F4E00AF3190006F124B18E0F599EFB40107EE38
:100F5E00B407037545007830124B58E545B40402CA
:100F6E00800302104CE53145307003852599AE3073
:100F7E00AF3174016F4E7003853799AE30AF317457
:100F8E00026F4E7003853999AE30AF3174036F4ED8
:100F9E007003853D99AE30AF3174046F4E7003858A
:100FAE003F99AE30AF3174056F4E7003854099AEE8
:100FBE0030AF3174066F4E7003854199AE30AF314C
:100FCE0074076F4E7003854299AE30AF3174086F5F
:100FDE004E7006900021E0F599AE30AF3174096F76
:100FEE004E7006900044E0F599AE30AF31740A6F42
:100FFE004E7003854399AE30AF31740B6F4E700354
:10100E00853E99AE30AF31740C6F4E7003854499A6
:10101E00AE30AF31740D6F4E7005900044E4F0AEFB
:10102E0030AF31740D6F4E70037599FC7830124BE2
:10103E0058AE30AF31740E6F4E7003754500E545F6
:10104E00B4051CAE30AF3190488E124B18E493F5B8
:10105E009974E06F4E70037545007830124B58E569
:10106E004664016005E546B40403020B2EC28E7E73
:10107E00107F00E53C124AF1E58D75F010A4FDAC31
:10108E00F0EF2DFDEE3CFCE58B75F01084FF7E003D
:10109E00ED2FFFEC3EFE8E268F27D28E90009CE029
:1010AE006056900022124AFF900022E0FCA3E0FD61
:1010BE00900024E0FAA3E0FBEDB5033CECB502385A
:1010CE00B216A208B34013A216B34008E5B5440405
:1010DE00F5B58006E5B554FBF5B5900024E0FEA30A
:1010EE00E0FF900026E0FCA3E0FDEF2DFDEE3CFCC2
:1010FE00900024ECF0A3EDF09000A9E060099000C0
:10110E00A9E0C394034002807A12447AA208B35035
:10111E0009900067E0C3944640028006900093E079
:10112E00F56AE56A75F005A4FFAEF09007B1EEF032
:10113E00A3EFF0900080E0C395394007E537C395E3
:10114E003850079007B1E4F0A3F0AE57AF589007B0
:10115E00B1E0FCA3E0FDEFD39DEE9C4004C2A18064
:10116E000B900067E0C394645002D2A19000A9E0F6
:10117E00B402099000C7E0C3940240028005A2A108
:10118E00B392A29000A9E0B4031C124576AE57AFFD
:10119E00589007B1E0FCA3E0FDEFD39DEE9C400418
:1011AE00D2A18002C2A1A2B6300901B35003021728
:1011BE0086A2B6300901B35003021786A2B6300BD1
:1011CE0001B350030216A07549000536A20DB3B344
:1011DE005013AE26AF27900012E0FCA3E0FDEDC346
:1011EE009FEC9E40030212D2E548B40330E536B4BC
:1011FE002405754801801FA21AB3401AE536C39420
:10120E002450069000447401F0E536D39424400631
:10121E007402900044F0753601D21A8044E548B449
:10122E000206754801753624E536B4240575360177
:10123E00802F900044E0701AE536C3942450069037
:10124E0000447401F0E536D39424400674029000F5
:10125E0044F09000B9E0B4020512036380037536C2
:10126E0001AE28AF29AC26AD27EF2DFDEE3CFC7468
:10127E0003FF1200858C288D2990009CE06043901E
:10128E000022E0FEA3E0FF90009CE08E048F05FF9D
:10129E0012008574018C068D07124AE3900026EE2B
:1012AE00F0A3EFF0900026E0F8A3E0900024C8F041
:1012BE00A3C8F0900022E4F0A3F0C216E5B554FBEB
:1012CE00F5B5802BAE28AF29AC26AD27EF2DFDEE60
:1012DE003CFC74018C068D07124AE38E288F29ACD4
:1012EE0026AD27EDD39488EC94134003120363E5E7
:1012FE0036B424107403900044F09000B9E0B402A8
:10130E0003120363AE2AAF2BAC26AD27EF2DFDEEF5
:10131E003CFC8C2A8D2BAE26AF27EFD39DEE9C4046
:10132E001190001AE0FAA3E0FBEBC394E8EA9403F1
:10133E004002800690001A124AFF900016E0FEA3AB
:10134E00E0FFAC26AD27EF2DFDEE3CFC900016EC39
:10135E00F0A3EDF09000B9E0B4021DAE26AF2774F5
:10136E0005124AF174038E048F05FF12008590005A
:10137E0012ECF0A3EDF08016AE26AF277403124ADE
:10138E00F17401124AE3900012EEF0A3EFF0900018
:10139E0004E0FEA3E0FF74E8D39F74FD9E401FACF3
:1013AE0026AD27EFD39DEE9C400D124B50900004BE
:1013BE00EEF0A3EFF08007900004E4F0A3F09000AD
:1013CE000CE0FEA3E0FF74E8D39F74FD9E401FACBB
:1013DE0026AD27EFD39DEE9C400D124B5090000C86
:1013EE00EEF0A3EFF0800790000CE4F0A3F0900075
:1013FE0006E0FEA3E0FF74E8D39F74FD9E401FAC91
:10140E0026AD27EFD39DEE9C400D124B509000065B
:10141E00EEF0A3EFF08007900006E4F0A3F090004A
:10142E000EE0FEA3E0FF74E8D39F74FD9E401FAC58
:10143E0026AD27EFD39DEE9C400D124B5090000E23
:10144E00EEF0A3EFF0800790000EE4F0A3F0900012
:10145E009CE07026E5366401600BE5366404600599
:10146E00E536B413028013A216B34008E5B5440462
:10147E00F5B58006E5B554FBF5B5C28E758D0075D4
:10148E008B00753C00752701752600D28EE536243B
:10149E000875F00984AFF07E00EF4E70759000165F
:1014AE00E0F8A3E0900014C8F0A3C8F0900014E098
:1014BE00FEA3E0FFEF4E600B7C7E7DE01249F38EC3
:1014CE00248F25900016E4F0A3F0AE24AF257428E7
:1014DE00BE00039F5010E53B2FFF50010E7401120A
:1014EE004AE38E248F2585253B9000C0E0A824B8C2
:1014FE00000DD395254008E525900041F080099018
:10150E0000C0E014900041F0E548600675250075B6
:10151E002400E536640B6005E536B41D099000A97C
:10152E00E060031241BC90003DE06536600790001C
:10153E003EE0B53603754A00A20E5003021608901F
:10154E000075E0B4015AE53F75F00584FF7E00900A
:10155E00056F124B18E0F533753200AE32AF339093
:10156E000073E0124AF174648E048F05FF12008539
:10157E0074C18C068D07124AF18E348F3590001887
:10158E00E0FEA3E0FFAC32AD3312000374648E04B0
:10159E008F05FF120085900018ECF0A3EDF0800F80
:1015AE00900073E075F0C1A4FFAEF08E348F35E578
:1015BE0039C394CC504275A71085F94F85FA507EE9
:1015CE00017F00E550124AF1E54F2FFF50010E8EBC
:1015DE00328F33AC34AD35EF2DFDEE3CFC8C348DBB
:1015EE0035D293D291E535F5FBE534F5FCE535F5CD
:1015FE00E9E534F5EA75A700D20EE548B40106E533
:10160E0036640B6002800F754B019000477401F039
:10161E00E5B54401F5B5E54870739000BCE0600D8A
:10162E009000C3E0A824B8000695254002803290B1
:10163E0000BCE0B40217900036E0653660079000FB
:10164E0037E0B53603754B03754400800CC2007548
:10165E004400900020E4F0A3F07409900044F08060
:10166E002C900036E065366007900037E0B5360303
:10167E00754B01900036E0B536069000477401F0C8
:10168E00900037E0B536067402900047F0A20BB317
:10169E009209A20BB330B601B350030217867549F7
:1016AE000190009CE07013A20BB34008E5B5440412
:1016BE00F5B58006E5B554FBF5B5A20B9209E536F6
:1016CE00D3944A4012D20DE536D3946E400974037A
:1016DE00900044F07536469000C4E0B40107E54230
:1016EE00C39414400280031203637446900067F0A3
:1016FE00A204300501B35017A204B34008E5B54467
:10170E0008F5B58006E5B554F7F5B5A2049205A225
:10171E0006300701B35017A206B34008E5B54402E0
:10172E00F5B58006E5B554FDF5B5A2069207E5427E
:10173E00C394415009740E900044F012036390005C
:10174E004EE0FE90004AE0C39E400990004AE0D36E
:10175E009406400974FB900044F01203639000530A
:10176E00E06015900053E0FE90004DE06E6009744D
:10177E00FE900044F0120363A210B3B35008900021
:10178E0038E0653660028077A202B35006A200B33D
:10179E00B34002806675A71085F94F85FA507E0119
:1017AE007F00E550124AF1E54F2FFF50010E8E32A9
:1017BE008F3390001EE0FCA3E0FDEF2DFDEE3CFC10
:1017CE008C348D35E535F5FBE534F5FCD293A2036B
:1017DE00B34002D2949000D5E0B4021CAE32AF33C7
:1017EE00AC55AD56EF2DFDEE3CFC8C348D35E5350C
:1017FE00F5EBE534F5ECD29475A700C210D211A228
:10180E0011B3B35008900039E0653660028077A2BC
:10181E0002B35006A200B3B34002806675A71085CE
:10182E00F94F85FA507E017F00E550124AF1E54FDF
:10183E002FFF50010E8E328F3390001EE0FCA3E07E
:10184E00FDEF2DFDEE3CFC8C348D35E535F5E9E5EF
:10185E0034F5EAD291A203B34002D2929000D5E0C1
:10186E00B4021CAE32AF33AC55AD56EF2DFDEE3C8F
:10187E00FC8C348D35E535F5EDE534F5EED292750B
:10188E00A700D210C211E54BB40816123AEBA21003
:10189E00B35005A211B340028004D210D211754B81
:1018AE001EE54BB407061238A3754B08E54BB4067C
:1018BE003D900018E0FEA3E0FFEF4E6006A208B3D5
:1018CE00B340028023AE51AF52900018E0FCA3E06B
:1018DE00FDEF2DFDEE3CFC8C518D52E536D394126E
:1018EE005006900018120039123675754B07E54BED
:1018FE00B405061234D5754B06E54BB40432900090
:10190E00AAE0902B5CF828287312316980121231EC
:10191E0069800D12331780081233C980031233C940
:0F2B5C0002191702191C02192102192602192B3E
:10192E0090008CE060051242A58002C204754B0542
:10193E00E54BB403028003021A2890008FE0600585
:10194E001243958002C2069000AAE0D39402403F53
:10195E0090007EE02403A824B80004952550099039
:10196E000080E0D3953950028008D20274089000AE
:10197E0044F090007EE0A824B80005D39525500BC6
:10198E00900080E02403C395395002C20280399042
:10199E00007EE02403A824B8000495255007E537FF
:1019AE00C3953840028008D2027408900044F0902B
:1019BE00007EE0A824B80005D395255009E538240B
:1019CE000FC395375002C2029000C4E07007E54283
:1019DE00C3941440028002D202A2024005754B0449
:1019EE00800A754B1E900020E4F0A3F0A208B340CD
:1019FE0029E53F75F00584FF7E0090056F124B18A8
:101A0E00E0C3946950051241F1800F9007A9E0F8E8
:101A1E00A3E09007A7C8F0A3C8F0E54BB40A028074
:101A2E0003021AE0900030E0C394465022C296742E
:101A3E0046900030F0900010E0FEA3E0FFAC26AD23
:101A4E0027EF2DFDEE3CFC90000CECF0A3EDF0909A
:101A5E00003AE0B4011DE559240AF5599007ABE0B0
:101A6E00FEA3E0FF740A2FFF50010E9007ABEEF0BD
:101A7E00A3EFF0855933753200900036E0F54F1222
:101A8E00009EE535900030F0900008E532F0A3E5B9
:101A9E0033F0E54F900031F0C2139007ABE0F53212
:101AAE00A3E0F533900036E0F54F12009EE5359039
:101ABE00002EF0900000E532F0A3E533F0E54F90F4
:101ACE00002FF0C212E548B40105754B0B8003756B
:101ADE004B0390002EE0B536028003021B72A21259
:101AEE00404F900000E0FEA3E0FFEF4E6021AE28D5
:101AFE00AF29900000E0FCA3E0FD120003740A8EF3
:101B0E00048F05FF120085900000ECF0A3EDF0901D
:101B1E00002FE0601A900000E0FEA3E0FFAC28ADBD
:101B2E0029EF2DFDEE3CFC900000ECF0A3EDF0D281
:101B3E0012AE26AF27900000E0FCA3E0FDEFC39DA0
:101B4E00EE9C4020D296C21274C890002EF09000E7
:101B5E0010E0FAA3E0FBEB2FFFEA3EFE900004EE4E
:101B6E00F0A3EFF0A212B3B3500790002EE0B536FB
:101B7E00028024D29674C890002EF0C212900010EB
:101B8E00E0FEA3E0FFAC26AD27EF2DFDEE3CFC9072
:101B9E000004ECF0A3EDF0900030E0B536028003C7
:101BAE00021C37A213404F900008E0FEA3E0FFEFA7
:101BBE004E6021AE28AF29900008E0FCA3E0FD1294
:101BCE000003740A8E048F05FF120085900008EC46
:101BDE00F0A3EDF0900031E0601A900008E0FEA353
:101BEE00E0FFAC28AD29EF2DFDEE3CFC900008EC9B
:101BFE00F0A3EDF0D213AE26AF27900008E0FCA3C1
:101C0E00E0FDEFC39DEE9C4020C2967446900030DE
:101C1E00F0C213900010E0FAA3E0FBEB2FFFEA3EB8
:101C2E00FE90000CEEF0A3EFF0A213B3B3500790AA
:101C3E000030E0B536028024C2967446900030F033
:101C4E00C213900010E0FEA3E0FFAC26AD27EF2DEF
:101C5E00FDEE3CFC90000CECF0A3EDF0AE26AF27B1
:101C6E00900004E0FCA3E0FDEFC39DEE9C400CD27F
:101C7E009590000474FFF0A374DCF0AE26AF2790AD
:101C8E00000CE0FCA3E0FDEFC39DEE9C400CC29562
:101C9E0090000C74FFF0A374DCF0E54BB40B0280E3
:101CAE0003021D6A900034E0C394465022C2A07411
:101CBE0046900034F0900010E0FEA3E0FFAC26AD9D
:101CCE0027EF2DFDEE3CFC90000EECF0A3EDF09016
:101CDE00003BE0B4011DE559240AF5599007ABE02D
:101CEE00FEA3E0FF740A2FFF50010E9007ABEEF03B
:101CFE00A3EFF0855933753200900037E0F54F129F
:101D0E00009EE535900034F090000AE532F0A3E530
:101D1E0033F0E54F900035F0C2159007ABE0F53289
:101D2E00A3E0F533900037E0F54F12009EE53590B5
:101D3E000032F0900002E532F0A3E533F0E54F906B
:101D4E000033F0C214E548B4010F75480074C89012
:101D5E00002EF074C8900032F0754B03900032E004
:101D6E00B536028003021DFCA214404F900002E023
:101D7E00FEA3E0FFEF4E6021AE28AF29900002E0F7
:101D8E00FCA3E0FD120003740A8E048F05FF1200FF
:101D9E0085900002ECF0A3EDF0900033E0601A9015
:101DAE000002E0FEA3E0FFAC28AD29EF2DFDEE3CD6
:101DBE00FC900002ECF0A3EDF0D214AE26AF27900B
:101DCE000002E0FCA3E0FDEFC39DEE9C4020D2A0FC
:101DDE00C21474C8900032F0900010E0FAA3E0FB39
:101DEE00EB2FFFEA3EFE900006EEF0A3EFF0A214FA
:101DFE00B3B35007900032E0B536028024D2A074FF
:101E0E00C8900032F0C214900010E0FEA3E0FFACC8
:101E1E0026AD27EF2DFDEE3CFC900006ECF0A3ED79
:101E2E00F0900034E0B536028003021EC1A21540C8
:101E3E004F90000AE0FEA3E0FFEF4E6021AE28AF08
:101E4E002990000AE0FCA3E0FD120003740A8E0440
:101E5E008F05FF12008590000AECF0A3EDF09000C4
:101E6E0035E0601A90000AE0FEA3E0FFAC28AD2931
:101E7E00EF2DFDEE3CFC90000AECF0A3EDF0D21538
:101E8E00AE26AF2790000AE0FCA3E0FDEFC39DEE67
:101E9E009C4020C2A07446900034F0C215900010F1
:101EAE00E0FAA3E0FBEB2FFFEA3EFE90000EEEF011
:101EBE00A3EFF0A215B3B35007900034E0B536028D
:101ECE008024C2A07446900034F0C215900010E039
:101EDE00FEA3E0FFAC26AD27EF2DFDEE3CFC9000FF
:101EEE000EECF0A3EDF0AE26AF27900006E0FCA3BB
:101EFE00E0FDEFC39DEE9C400CD29790000674FF60
:101F0E00F0A374DCF0AE26AF2790000EE0FCA3E049
:101F1E00FDEFC39DEE9C400CC29790000E74FFF037
:101F2E00A374DCF0E54BB402028003022077123F6B
:101F3E005412406B1241589007A7E0FEA3E0FF74C5
:101F4E000A124AF1900014E0FCA3E0FD74098F021E
:101F5E00FF1200858D078C038E048A058B061249AD
:101F6E00F39007ABEEF0A3EFF074F0BE00039F50BA
:101F7E000B74F09007ABF8E4F0E8A3F09007ABE039
:101F8E00FEA3E0FFE5592FFF50010E9007ABEEF0D8
:101F9E00A3EFF0900014E0FCA3E0FD7478D39D74E1
:101FAE00059C401F9007B6E08C068D07124AF1740F
:101FBE005A8E048F05FF120085900010ECF0A3EDF1
:101FCE00F0802F900014E0FEA3E0FF74098E048FC2
:101FDE0005FF1200859007B6E08C068D07124AF1B8
:101FEE00740A8E048F05FF120085900010ECF0A38A
:101FFE00EDF09000C5E0B4025C9007A7E0FEA3E010
:10200E00FF740A124AF1900014E0FCA3E0FD74097B
:10201E008F02FF1200858D078C038E048A058B06B6
:10202E001249F39007ABEEF0A3EFF07478BE000305
:10203E009F500B74789007ABF8E4F0E8A3F090078C
:10204E00ABE0FEA3E0FFE5592FFF50010E9007AB6A
:10205E00EEF0A3EFF0900047E0B40103754B0A9049
:10206E000047E0B40203754B0BE54BB4012590001D
:10207E00DCE0902B6BF8282873123CF28012123C95
:10208E00F2800D123D7C8008123E288003123E28FD
:0F2B6B0002208702208C02209102209602209BDC
:10209E00754B029000C7E0B4020280030221B99092
:1020AE00006AE0D3953E506490006AE0F404253E49
:1020BE00FE9000CAE08E00F5F0E884FF7E008F4FA0
:1020CE00EFC39410500CEF854FF0A4FDACF08D4F84
:1020DE008003754FFF90006AE0D3954F400B900040
:1020EE006AE0C3954FF54C8003754C009000E5E017
:1020FE00D3954C40069000E5E0F54C9000E6E0C329
:10210E00954C50069000E6E0F54C807190006AE028
:10211E00C3953EFE9000CAE08E00F5F0E884FF7E87
:10212E00008F4FEFC39410500CEF854FF0A4FDAC11
:10213E00F08D4F8003754FFF854F33753200900041
:10214E006AE02533FFAE3250010E8E328F3374FFAC
:10215E00BE0009D39F400585334C8003754CFF901C
:10216E0000E5E0D3954C40069000E5E0F54C90007C
:10217E00E6E0C3954C50069000E6E0F54CA208B39D
:10218E00B350099000D2E0D3954D5002800A7407E7
:10219E00900044F0C2A2801375A710E5CDC3954CF4
:1021AE004004C2A28002D2A275A700E54AC39409D8
:1021BE0040030228E8A2EDB350030228E8C2EDE581
:1021CE004A600302235C900078E0700302234B9078
:1021DE0000AEE0B4010280030222AB7E017F00E577
:1021EE00BE124AF1E5BD2FFF50010E8E328F339095
:1021FE000078E0B401187410124AF190006EE08E6F
:10220E00048F05FF120085ED90003FF0802CAE325A
:10221E00AF337410124AF190006EE08E048F05FFFA
:10222E0012008590003FE02DFD50010C74018C06CC
:10223E008D07124AE3EF90003FF0E54360089000EF
:10224E00D4E06402600280219000D6E0B4011A90BE
:10225E00003FE075F0E7A4FFAEF0E5438E048F0576
:10226E00FF120085ED90003FF090003FE0FE9000E1
:10227E0040E0D39E4004D2188002B21890003FE096
:10228E00900040F09000AAE064016006A218B3B37B
:10229E004002800690003FE0F537022349D2187EB7
:1022AE00017F00E5BE124AF1E5BD2FFF50010E8EF3
:1022BE00328F33900078E0B401187410124AF19006
:1022CE00006EE08E048F05FF120085ED90003FF04A
:1022DE00802CAE32AF337410124AF190006EE08E45
:1022EE00048F05FF12008590003FE02DFD50010C7C
:1022FE0074018C068D07124AE3EF90003FF0E54320
:10230E0060089000D4E06402600280219000D6E064
:10231E00B4011A90003FE075F0E7A4FFAEF0E5437C
:10232E008E048F05FF120085ED90003FF09000AAFD
:10233E00E06401600690003FE0F5378003753700DA
:10234E00900074E07005754A01800375BB18E54A6C
:10235E00B4010280030224FE900074E07003022494
:10236E00ED7E017F00E5BE124AF1E5BD2FFF500163
:10237E000E8E328F339000BAE0B4010F7E0F7FFFC6
:10238E00AC32AD33124B508E328F339000DFE0B44F
:10239E000245AE32AF3390002AE0FCA3E0FDEDD350
:1023AE009FEC9E400A90002AE532F0A3E533F0AE92
:1023BE0032AF3390002CE0FCA3E0FDEFD39DEE9CFA
:1023CE00400A90002CE532F0A3E533F0AE32AF3385
:1023DE007404124AE38F399000DFE0704CAE32AFD6
:1023EE003390002AE0FCA3E0FDEFD39DEE9C400964
:1023FE00124B508E328F338006753300753200AE1D
:10240E0032AF337410124AF190006BE08E048F05D8
:10241E00FF1200858C328D337400D39D74019C4065
:10242E000585333980037539FF9000AAE0B40102A7
:10243E0080030224EBA208B3B3500E90007EE0A8F6
:10244E0024B80005D3952550030224E090007FE0C8
:10245E0075F019A4FFAEF09000C2E08E048F05FF58
:10246E001200859000BBE08539F0A4FFAEF07464D5
:10247E008D028C038E048F05FF120085EA2DFDEB75
:10248E003CFC8C328D33E543600F9000D4E0B402F7
:10249E00089000D6E0640160028017AE32AF33744C
:1024AE00E7124AF1E5438E048F05FF1200858C3248
:1024BE008D3390003FE0A832B8000AD39533400523
:1024CE00853337800BA218B3400690003FE0F537F6
:1024DE00800BA218B3400690003FE0F537800375DD
:1024EE003900900077E07005754A02800375BB19BC
:1024FE00E54AB4020280030225B9900077E070032A
:10250E000225A8E536D3941240030225A690002892
:10251E00E0FEA3E0FFE53D124B48900028EEF0A34D
:10252E00EFF07E017F00E5BE124AF1E5BD2FFF50B0
:10253E00010E8E328F339000E4E07013740A124A4B
:10254E00F174518E048F05FF1200858D3D8019AEFA
:10255E0032AF33740A124AF18F048E057E017F95D5
:10256E00CDCCCD1249F38F3DE53DD3946440037538
:10257E003D64900028E0FEA3E0FFE53D2FFF5001F3
:10258E000E900028EEF0A3EFF090007BE0048E0496
:10259E008F05FF1200858D3D8003753D329000C77B
:1025AE00E07005754A03800375BB13E54AB4035EFC
:1025BE009000C7E060477E017F00E5BE124AF1E55C
:1025CE00BD2FFF50010E8E328F337404124AE38FEB
:1025DE003E9000C9E0853EF0A4FDACF07464FF129D
:1025EE0000858D3E9000C8E0853EF0A4FFAEF074ED
:1025FE00FF8E048F05FF1200858D4D8003753E0002
:10260E00900075E07005754A04800375BB17E54AA6
:10261E00B4040280030226BA900075E0B4017C7EF9
:10262E00017F00E5BE124AF1E5BD2FFF50010E7489
:10263E0004124AE38E328F33900042E06012900013
:10264E0042E01490479C93A832B80006953340029E
:10265E008006900042E014F0900042E0C394775060
:10266E0013900042E00490479C93A832B80005D323
:10267E00953350028006900042E004F0900042E054
:10268E00FE90009BE08E0088F0A4FFAEF074648E86
:10269E00048F05FF1200858D3F8003753F0090006B
:1026AE0076E07005754A05800375BB16E54AB405DC
:1026BE0002800302274D900076E0B4017C7E017FFC
:1026CE0000E5BE124AF1E5BD2FFF50010E74041253
:1026DE004AE38E328F33900043E06012900043E065
:1026EE001490481593A832B8000695334002800620
:1026FE00900043E014F0900043E0C39477501390A1
:10270E000043E00490481593A832B80005D39533E2
:10271E0050028006900043E004F0900043E0FE90EB
:10272E0000A1E08E0088F0A4FFAEF074648E048FDA
:10273E0005FF1200858D40800375400075BB1FE5B7
:10274E004AB406337E017F00E5BE124AF1E5BD2F85
:10275E00FF50010E8E328F337409124AF174E68ED9
:10276E00048F05FF1200858D4290007DE070057587
:10277E004A07800375BB15E54AB407028003022899
:10278E008F90007DE0700302287E7E017F00E5BE03
:10279E00124AF1E5BD2FFF50010E8E328F337404B5
:1027AE00124AE38F4190007DE0B401159000D1E014
:1027BE008541F0A4FFAEF07407124AE3EF9007B420
:1027CE00F090007DE0B402159000D1E08541F0A4B8
:1027DE00FFAEF07407124AE3EF9007B3F090007D5E
:1027EE00E0B40302800302287C9000BEE0701CE57A
:1027FE0041C3940A5002D201E541D394644002C20F
:10280E000190009DE0900069F0806390009DE07063
:10281E00349000D1E08541F0A4FFAEF074FF8E0439
:10282E008F05FF120085ED900069F0AE24AF257480
:10283E001EBE0006D39F4002D201E539D394E54077
:10284E0002C2018029E541C3940A500DAE24AF2582
:10285E00741EBE0004D39F50028002D201E539D30C
:10286E0094E54002C20190009DE0900069F0800363
:10287E007541009000D4E07005754A08800375BB61
:10288E0014E54AB408509000D4E060397E017F0010
:10289E00E5BE124AF1E5BD2FFF50010E8E328F3389
:1028AE00EFD39421EE940E40057543FF8015AE32A2
:1028BE00AF337410124AF174E38E048F05FF1200C9
:1028CE00858D438003754300900078E0600575BBED
:1028DE001A800375BB18054AD2ECAE26AF27EFD38C
:1028EE009410EE94275003022B59C20D7536469064
:1028FE0000B9E070057548028003754803C293C2A3
:10290E0094C291C292C287C290E5B554EFF5B5E577
:10291E00B554DFF5B5C296C295C2A0C297C2A2C287
:10292E00A1E5B5547FF5B5E5B554BFF5B5A219B31C
:10293E004008E5B54404F5B58006E5B554FBF5B59C
:10294E00A20FB3500EE539D394334007E539C39443
:10295E00CC4002806EE5B54401F5B5744690006733
:10296E00F0900073E075F064A4FFAEF08E348F35F6
:10297E007402BE000AD39F40067535027534007589
:10298E00A71085F94F85FA507E017F00E550124A57
:10299E00F1E54F2FFF50010E8E328F33AC34AD3533
:1029AE00EF2DFDEE3CFC8C348D35D293D291E53576
:1029BE00F5FBE534F5FCE535F5E9E534F5EA75A703
:1029CE0000D20FE539C3941A5002C20F9000127450
:1029DE00FFF0A374DCF090009AE0900018F8E4F099
:1029EE00E8A3F0C212C21474C890002EF074C890FE
:1029FE000032F090001074FFF0A374DCF090000C25
:102A0E0074FFF0A374DCF090000E74FFF0A374DC7E
:102A1E00F090000474FFF0A374DCF090000674FFD5
:102A2E00F0A374DCF0C210C2117525007524007578
:102A3E003B00C208756B00900020E4F0A3F0754BCC
:102A4E001E9007A9E0FEA3E0FF7403124AF1740181
:102A5E00124AE39007A7EEF0A3EFF090008CE0602F
:102A6E00051242A58002C20490008FE06005124359
:102A7E00958002C206A204300501B35017A204B31A
:102A8E004008E5B54408F5B58006E5B554F7F5B54B
:102A9E00A2049205A206300701B35017A206B34056
:102AAE0008E5B54402F5B58006E5B554FDF5B5A2C9
:102ABE00069207C203752B00752A0090001AE4F0E7
:102ACE00A3F090007BE075F032A4FFAEF0900028EA
:102ADE00EEF0A3EFF0900016E4F0A3F0C21A90000F
:102AEE0068E0C3943C5019758D6E758B00753C0271
:102AFE00E54AB40909900068E004F0754A00803B8D
:102B0E00E54AB40903754A00752700752600758DD0
:102B1E0000758B00753C00900067E0C3946450080C
:102B2E00900067E004F080067464900067F09000F7
:102B3E0067E0B46406E5B554FEF5B5E542C39441CD
:0E2B4E005009740E900044F0120363020B2E27
:104724000000010001400160018001A001C001E01E
:1047340002000300039603B603D603F40400050045
:1047440005180530054805600578059005A805C0DD
:10475400060006140628063C066E068C00FF013F80
:10476400015F017F019F01BF01DF01FF02FF03958C
:1047740003B503D503F303FF04FF0517052F05470E
:10478400055F0577058F05A705BF05FF06130627F7
:10479400063B066F068B06A9DAD8D7D5D4D2D0CF7C
:1047A400CDCBC9C7C6C4C2C0BEBCBAB8B5B3B1AF1D
:1047B400ADABA8A6A4A2A09D9B99969492908D8B34
:1047C40089878482807E7C79777573716F6D6B695C
:1047D400676563615F5D5B5957565452504F4D4B4B
:1047E4004A4847454442413F3E3C3B3A39373635D7
:1047F400343231302F2E2D2C2B2A292827262525FB
:104804002423222121201F1E1E1D1C1C1B1A1A19C1
:1048140019EEECEBEAE9E8E7E5E4E3E1E0DEDDDB11
:10482400D9D8D6D4D2D0CECCCAC8C6C3C1BFBCBADC
:10483400B7B5B2B0ADABA8A5A3A09D9B9895929037
:104844008D8A8785827F7D7A7775726F6D6A6865D8
:1048540063615E5C5A575553514F4D4B494745432D
:1048640042403E3C3B393836353332312F2E2D2BE6
:104874002A292827262524232221201F1E1D1D1C0A
:0A4884001B1A1A191818171616153A
:102B7A00750B00750A00AE0AAF0BAC08AD09EDC3C0
:102B8A009FEC9E401674FF12007575CF01780B7486
:102B9A000126F6500418E436F650DB2290003CE099
:102BAA00B4AA1C90076FE0B43C159007AFE0FEA3EF
:102BBA00E0FFEF4E6009741EBE0004D39F5003026B
:102BCA002CD475350075340075F8099007AFE0FE0E
:102BDA00A3E0FF74076F4E6006740E6F4E700674A2
:102BEA003A90076FF09007AFE0FEA3E0FF7408BECB
:102BFA00001ED39F401A7E017F089007AFE0FCA316
:102C0A00E0FD1DBDFF011C1200038E328F33801FB1
:102C1A009007AFE0FEA3E0FF7408124B488F048EC2
:102C2A00057E017F08CDCCCD1200038E328F33AEE4
:102C3A0034AF35740CD39F74019E5003022CCFA27B
:102C4A00F9B3407EE5354534700375A382AE34AFDF
:102C5A003574016F4E700375A300AE34AF3574023C
:102C6A006F4E700D9007B0E075F002A4FDACF08DC8
:102C7A00A3AE34AF3574036F4E700375A300AE3440
:102C8A00AF357403BE00039F5013AC32AD33ED2F42
:102C9A00FFEC3EFE90006B124B18E0F5A3AE34AF8A
:102CAA0035EFB40B09EEB401057414120075AE3495
:102CBA00AF35EFB40B07EEB4010375F80D78341293
:102CCA004B58022C3990003CE4F0227535007534DB
:102CDA000075F8099007AFE0FEA3E0FF7408BE0094
:102CEA001ED39F401A7E017F089007AFE0FCA3E045
:102CFA00FD1DBDFF011C1200038E328F33801F9011
:102D0A0007AFE0FEA3E0FF7408124B488F048E055C
:102D1A007E017F08CDCCCD1200038E328F33AE34C4
:102D2A00AF357411D39F74019E5003022E05A2F988
:102D3A00B35003022E02E5354534700375A3D2AEB3
:102D4A0034AF3574016F4E700375A300AE34AF35DE
:102D5A0074026F4E700D9007B0E075F002A4FDACDE
:102D6A00F08DA3AE34AF3574036F4E700375A300B4
:102D7A00AE34AF3574046F4E700375A300AE34AF32
:102D8A003574056F4E700375A300AE34AF35740603
:102D9A006F4E700375A300AE34AF3574076F4E7073
:102DAA000375A300AE34AF3574086F4E700375A374
:102DBA0000AE34AF357408BE00039F5016AC32AD76
:102DCA0033ED2FFFEC3EFE900066124B18E5A3F0A0
:102DDA0075A300AE34AF35EFB41009EEB401057433
:102DEA0014120075AE34AF35EFB41007EEB4010318
:102DFA0075F80D7834124B58022D28227535007556
:102E0A00340075F809AE34AF357417BE0004D39F89
:102E1A005003022EDEA2F9B35003022EDBE535453C
:102E2A0034700375A3D2AE34AF3574016F4E70039C
:102E3A0075A300AE34AF3574026F4E700D9007B0B3
:102E4A00E075F002A4FDACF08DA3AE34AF35740387
:102E5A006F4E700375A300AE34AF3574046F4E70B5
:102E6A000375A300AE34AF3574056F4E700375A3B6
:102E7A0000AE34AF3574066F4E700375A300AE34DE
:102E8A00AF3574076F4E700375A300AE34AF357457
:102E9A00086F4E700375A300AE34AF357408BE00D8
:102EAA00039F500C900050124B18E5A3F075A30035
:102EBA00AE34AF3574166F4E70057414120075AEC9
:102ECA0034AF3574166F4E700375F80D7834124BA3
:102EDA0058022E0F2290003CE0B4AB028003022F6E
:102EEA007975350075340075F809AE34AF3574124A
:102EFA00BE007CD39F4078A2F9B34070E5354534D3
:102F0A00700375A382AE34AF3574016F4E700375CA
:102F1A00A300AE34AF3574026F4E700D9007B0E067
:102F2A0075F002A4FDACF08DA3AE34AF3574036F17
:102F3A004E700375A300AE34AF357403BE00039F11
:102F4A005009900055124B18E0F5A3AE34AF357412
:102F5A00116F4E70057414120075AE34AF357411CA
:102F6A006F4E700375F80D7834124B58022EF42206
:102F7A00900045E4F074649007AFF8E4F0E8A3F039
:102F8A00122E0674C89007AFF8E4F0E8A3F0900098
:102F9A005CE0B4371A900059E0900050F090005A63
:102FAA00E0900051F090005BE0900052F080469073
:102FBA0000457401F074659007AFF8E4F0E8A3F0F7
:102FCA00122E0674C89007AFF8E4F0E8A3F0900058
:102FDA005CE0B4371A900059E0900050F090005A23
:102FEA00E0900051F090005BE0900052F08006748F
:102FFA0002900045F0900046E4F074669007AFF83E
:10300A00E4F0E8A3F0122E0674C89007AFF8E4F0D3
:10301A00E8A3F090005BE0B43712900059E090000A
:10302A004AF090005AE0900053F08076900046747F
:10303A0001F074679007AFF8E4F0E8A3F0122E06E7
:10304A0074C89007AFF8E4F0E8A3F090005BE0B42E
:10305A003712900059E090004AF090005AE0900030
:10306A0053F0803E7402900046F074689007AFF8FF
:10307A00E4F0E8A3F0122E0674C89007AFF8E4F063
:10308A00E8A3F090005BE0B43712900059E090009A
:10309A004AF090005AE0900053F0800674039000C2
:1030AA0046F022E55C2533FFAE3250010E90006FE8
:1030BA00124B18E0F55DE55C2533FFAE3250010E88
:1030CA000FBF00010E90006F124B18E0F55E856489
:1030DA0060E55DB55E05855D5C8041E55ED3955D25
:1030EA00401DE55EC3955D855FF0A4FFAEF0E56027
:1030FA008E048F05FF120085ED255DF55C801DE5C8
:10310A005DC3955E855FF0A4FFAEF0E5608E048F27
:10311A0005FF120085EDF404255DF55C22E55ED31A
:10312A00955D401DE55EC3955D855FF0A4FFAEF039
:10313A00E5608E048F05FF120085ED255DF55C8044
:10314A001DE55DC3955E855FF0A4FFAEF0E5608E78
:10315A00048F05FF120085EDF404255DF55C22E578
:10316A003775F00484FF7E008F5CE53775F00484C0
:10317A00ADF07C008D5F756404753201753300E52E
:10318A005CC3943F50051230AD80069001AEE0F565
:10319A005C855C52755100900041E075F020A4FFF7
:1031AA00AEF09000C0E08E048F05FF1200858D5CA2
:1031BA009000A8E0D39537500302326F9000CCE01C
:1031CA00D395374010ED9001AF124B2DE0F55475B1
:1031DA00530002326C900097E0D395374043E55C88
:1031EA009001AF124B2DE0F55DE55C9001CF124BDB
:1031FA002DE0F55E9000CCE0F4042537F55F9000F1
:10320A0097E0FE9000CCE0F4042EF560E55DB55E33
:10321A0005855D5C8003123127855C5475530080F7
:10322A0041E55C9001CF124B2DE0F55DE55C900124
:10323A00EF124B2DE0F55E900097E0F4042537F588
:10324A005F9000A8E0FE900097E0F4042EF560E598
:10325A005DB55E05855D5C8003123127855C54751A
:10326A0053000233169000CFE0D395375011E55C36
:10327A0090022F124B2DE0F554755300023316902D
:10328A000098E0D395375043E55C90020F124B2D1E
:10329A00E0F55DE55C90022F124B2DE0F55E9000A3
:1032AA0098E0F4042537F55F9000CFE0FE9000988F
:1032BA00E0F4042EF560E55DB55E05855D5C80038E
:1032CA00123127855C547553008041E55C9001EF0B
:1032DA00124B2DE0F55DE55C90020F124B2DE0F5E7
:1032EA005E9000A8E0F4042537F55F900098E0FEB0
:1032FA009000A8E0F4042EF560E55DB55E05855DF5
:10330A005C8003123127855C54755300229000E0DB
:10331A00E0F561756411753202753300AE24AF258C
:10332A00E56175F00FA4FDACF0EDD39FEC9E402152
:10333A00E5618E048F05FF120085ED75F010A4FF7C
:10334A00AEF0E53775F01184FD7C00ED2FF5628053
:10335A000EE53775F01184FF7E00EF24F0F56285E3
:10336A00625CE53775F01184AFF07E008F5F123032
:10337A00AD855C63AE24AF259000E0E075F00FA444
:10338A00FDACF0EDD39FEC9E4028753202753310E8
:10339A0085625C1230AD85635D855C5EAE24AF25C7
:1033AA00E5618E048F05FF124B0C8D5F85616012FB
:1033BA003127855C5275510075546475530022900B
:1033CA0000E0E0F561756411753202753300AE24D0
:1033DA00AF25E56175F00FA4FDACF0EDD39FEC9E2F
:1033EA004021E5618E048F05FF120085ED75F0100E
:1033FA00A4FFAEF0E53975F01184FD7C00ED2FF5E0
:10340A0062800EE53975F01184FF7E00EF24F0F535
:10341A006285625CE53975F01184AFF07E008F5FDA
:10342A001230AD855C63AE24AF259000E0E075F004
:10343A000FA4FDACF0EDD39FEC9E402875320275C7
:10344A00331085625C1230AD85635D855C5EAE24A7
:10345A00AF25E5618E048F05FF124B0C8D5F8561E8
:10346A0060123127855C527551009000AAE0B404BD
:10347A0053E53775F00484FF7E008F5CE53775F0FD
:10348A000484ADF07C008D5F756404753201753378
:10349A0000E55CC3943F50051230AD80069001AE42
:1034AA00E0F55CAE51AF52E55C124AF174648E04E9
:1034BA008F05FF120085AE51AF52EF2DFDEE3CFC99
:1034CA008C518D5275546475530022900075E0B486
:1034DA000146E53F75F00584FF7E008F5CE53F7588
:1034EA00F00584ADF07C008D5F7564057532057555
:1034FA003300E55CC3941750051230AD8006900581
:10350A0086E0F55CAE53AF54E55C2FFF50010E74B4
:10351A0064124B488E538F54900076E0B40146E50E
:10352A004075F00584FF7E008F5CE54075F00584E8
:10353A00ADF07C008D5F756405753205753348E51D
:10354A005CC3941750051230AD80069005CEE0F5A5
:10355A005CAE53AF54E55C2FFF50010E7464124BFE
:10356A00488E538F54900085E0B40249E542C394D3
:10357A004175F00584FF7E008F5CE54275F0058495
:10358A00ADF07C008D5F756405753206753300E514
:10359A005CC3941350051230AD8006900682E0F5A4
:1035AA005CAE53AF54E55C2FFF50010E7464124BAE
:1035BA00488E538F549000C7E0B40202800302364B
:1035CA0074E53775F01584FF7E008F5CE53775F07A
:1035DA001584ADF07C008D5F756415753203753303
:1035EA00F4E55CC3940B50051230AD800690046E6E
:1035FA00E0F55CE55C75F0FFA4FFAEF09000C8E072
:10360A008E048F05FF120085ED90006AF0E53E7585
:10361A00F078A4FFAEF074FF8E048F05FF120085C8
:10362A008C328D3374028C068D07124AE38F5CACA0
:10363A0032AD337404FF124B0C8D5F75640475321E
:10364A000675336EE55CC3941D50051230AD8006D5
:10365A009006FAE0F55CAE53AF54E55C2FFF5001DB
:10366A000E7464124B488E538F542290007DE0B43E
:10367A0001179007B4E02554FFAE5350010E900095
:10368A00D1E0124B488E538F5490007DE0B403165C
:10369A00A201B3B35010900069E0C39405A824B8FE
:1036AA00000695254002801090009FE02554FFAE49
:1036BA005350010E8E538F54900077E0B40202806B
:1036CA00030238A290007AE0602FE53FD3941E40AF
:1036DA002890001AE0FEA3E0FF9000B5E075F00321
:1036EA00A4FDACF0EFD39DEE9C400E9000D9E0A86B
:1036FA0024B80005D3952550030238A29000C2E0F1
:10370A008537F0A4FFAEF07405124AF17407124A25
:10371A00E38E328F33900081E0A824B80004952507
:10372A005012900082E075F002A4FDACF0EFC39D48
:10373A00EE9C40030238A2E53775F00B84FF7E0049
:10374A009005FF124B18FEE0FFEE900079E0FEEFC5
:10375A008E0088F0A4FFAEF074648E048F05FF1209
:10376A0000858C328D33900041E075F018A4FFAECD
:10377A00F09000C0E08E048F05FF1200858C068D44
:10378A0007900617124B18AE32AF33E0124AF174A3
:10379A00648E048F05FF1200858C328D33E53DA8B7
:1037AA0032B80077D395334072E53DC39533FFE4D1
:1037BA009532FE8E328F337428BE00039F500C75EB
:1037CA003328753200740D900044F0AE32AF339056
:1037DA00007AE0124AF174288E048F05FF120085E0
:1037EA008C328D33AE51AF52740A8E048F05FF129C
:1037FA0000858D068C07AC32AD33CFCECF120003D5
:10380A00740A8E048F05FF1200858C328D33AE51F7
:10381A00AF52124B508E518F52807DE53DA832B87F
:10382A00000495335072AE32AF33E53D124B488EE9
:10383A00328F337428BE00039F500C7533287532BB
:10384A0000740D900044F0AE32AF3390007AE0126B
:10385A004AF174288E048F05FF1200858C328D334D
:10386A00AE51AF52740A8E048F05FF1200858D0681
:10387A008C07AC32AD33CFCECF120003740A8E045C
:10388A008F05FF1200858C328D33AE51AF52EF2D6A
:10389A00FDEE3CFC8C518D5222AE51AF52AC53AD71
:1038AA005412000374648E048F05FF1200858C5134
:1038BA008D52900072E08C068D07124AF174648E64
:1038CA00048F05FF1200858C518D52A2084017AE55
:1038DA0024AF257405BE00039F5002D208E539D3F0
:1038EA0094CC4002D2029000D4E0B402089000D6F0
:1038FA00E0640160028017AE51AF52E543124AF10B
:10390A0074E78E048F05FF1200858C518D5290004A
:10391A0094E05402601B90008BE0A824B80012D3F4
:10392A009525400DA208B3B35007E539C3949A40D0
:10393A00028028AE5AAF5B900089E075F002A4FDC0
:10394A00ACF0EF2DFDEE3CFC74022DFD50010CE5B0
:10395A0039BC0007D39D400375680185395B755AE8
:10396A0000E56870030239F99000E7E0C395684002
:10397A0070E53F75F00584FF7E0090056F124B18C5
:10398A00E0F533753200AE32AF33900099E0124A57
:10399A00F174648E048F05FF1200858C348D359086
:1039AA0000E7E004C395688C068D07124AF190007F
:1039BA00E7E08E048F05FF1200858C348D35900068
:1039CA008AE08C068D07124AF1740A8E048F05FF6D
:1039DA00120085AE51AF52EF2DFDEE3CFC8C518D9D
:1039EA005205689000E7E0C3956850037568009037
:1039FA000094E05401601B900088E0A824B80012EB
:103A0A00D39525400DA208B3B35007E537C394CC2C
:103A1A0040028025900086E075F003A4FFAEF0E531
:103A2A00652FFF50010E74032FFF50010EE537BEBC
:103A3A000007D39F4003756901853765E5697003FF
:103A4A00023AD49000E8E0C395694070E53F75F00A
:103A5A000584FF7E0090056F124B18E0F53375322E
:103A6A0000AE32AF33900099E0124AF174648E04CA
:103A7A008F05FF1200858C348D359000E8E004C371
:103A8A0095698C068D07124AF19000E8E08E048F42
:103A9A0005FF1200858C348D35900087E08C068DE9
:103AAA0007124AF1740A8E048F05FF120085AE517F
:103ABA00AF52EF2DFDEE3CFC8C518D520569900002
:103ACA00E8E0C395695003756900900099E0A85130
:103ADA00B8000495525009900099E0F552755100CA
:103AEA00229000D5E0B401028003023BF6A208B39B
:103AFA005003023BF49000A0E0B40168AE51AF520B
:103B0A00AC24AD25120003743C8E048F05FF12000D
:103B1A00859000B0E0BC00109D400D9000B2E0A876
:103B2A0051B8000495525002D203AE51AF52AC24A0
:103B3A00AD25120003743C8E048F05FF1200859098
:103B4A0000B0E0C3940ABC0015D39D40119000B2A6
:103B5A00E0C39405A851B80005D3955250028002DB
:103B6A00C2038068AE51AF52AC24AD251200037473
:103B7A00788E048F05FF1200859000B0E0BC00101B
:103B8A009D400D9000B2E0A851B80004955250042F
:103B9A00D2038038AE51AF52AC24AD251200037463
:103BAA00788E048F05FF1200859000B0E0C3940A56
:103BBA00BC0015D39D40119000B2E0C39405A851F2
:103BCA00B80005D3955250028002C203A203B34043
:103BDA0019AE51AF529000B1E0124AF174648E04EA
:103BEA008F05FF1200858C518D528002C20390000E
:103BFA00D5E0B40258E53775F00884FF7E008F5C83
:103C0A00E53775F00884ADF07C008D5F7564087542
:103C1A0032017533E0E55CC3943F50051230AD8044
:103C2A000690026EE0F55CE55C75F05EA4FFAEF00E
:103C3A00740A8E048F05FF1200858C558D56740206
:103C4A00BC000AD39D4006755602755500A200B302
:103C5A004006A202B3B35009900020E4F0A3F0801A
:103C6A0024AE51AF527400D39F74019E400C900051
:103C7A0020E551F0A3E552F0800B74FF900020F884
:103C8A00E4F0E8A3F09000B7E0D394024006A2085B
:103C9A00B3B34002800DAE51AF527402124AF18E94
:103CAA00518F529000A0E0B4010DAE51AF52740290
:103CBA00124AF18E518F52AE51AF52745E124AF1CE
:103CCA00740A8E048F05FF1200858C518D5274027E
:103CDA00BC000AD39D400675520275510090001E21
:103CEA00E551F0A3E552F022900041E090036F12F3
:103CFA004B2DE0F566756764900041E0FE9000ABDD
:103D0A00E0D39E4037E53775F00884FF7E008F5C6C
:103D1A00E53775F00884ADF07C008D5F7564087531
:103D2A003203753396E55CC3941F50051230AD809B
:103D3A0006900424E0F55C855C678035E53775F00C
:103D4A000884FF7E008F5CE53775F00884ADF07C4F
:103D5A00008D5F7564087532037533B6E55CC394EC
:103D6A001F50051230AD8006900444E0F55C855C76
:103D7A0067229000E1E0F5617564117532047533CC
:103D8A0000AE24AF25E56175F00FA4FDACF0EDD3CC
:103D9A009FEC9E4021E5618E048F05FF120085EDA0
:103DAA0075F010A4FFAEF0E53775F01184FD7C00C4
:103DBA00ED2FF562800EE53775F01184FF7E00EF76
:103DCA0024F0F56285625CE53775F01184AFF07E08
:103DDA00008F5F1230AD855C63AE24AF259000E1A1
:103DEA00E075F00FA4FDACF0EDD39FEC9E40287572
:103DFA00320475331085625C1230AD85635D855C73
:103E0A005EAE24AF25E5618E048F05FF124B0C8D43
:103E1A005F856160123127855C6675676422900050
:103E2A00E1E0F561756411753204753300AE24AFB3
:103E3A0025E56175F00FA4FDACF0EDD39FEC9E4033
:103E4A0021E5618E048F05FF120085ED75F010A43F
:103E5A00FFAEF0E53975F01184FD7C00ED2FF562B7
:103E6A00800EE53975F01184FF7E00EF24F0F562CB
:103E7A0085625CE53975F01184AFF07E008F5F12C0
:103E8A0030AD855C63AE24AF259000E1E075F00F9C
:103E9A00A4FDACF0EDD39FEC9E4028753204753337
:103EAA001085625C1230AD85635D855C5EAE24AFC1
:103EBA0025E5618E048F05FF124B0C8D5F856160CD
:103ECA00123127855C667567649000DCE0B404797A
:103EDA00900041E0FE9000ABE0D39E4037E5377595
:103EEA00F00884FF7E008F5CE53775F00884ADF03A
:103EFA007C008D5F756408753203753396E55CC383
:103F0A00941F50051230AD8006900424E0F55C85BC
:103F1A005C678035E53775F00884FF7E008F5CE5C5
:103F2A003775F00884ADF07C008D5F7564087532D2
:103F3A00037533B6E55CC3941F50051230AD800695
:103F4A00900444E0F55C855C6722900075E0B4015A
:103F5A003BE53F75F00584FF7E008F5CE53F75F019
:103F6A000584ADF07C008D5F756405753205753387
:103F7A0018E55CC3941750051230AD800690059E73
:103F8A00E0F55CE567255CC39464F567900076E02C
:103F9A00B4013BE54075F00584FF7E008F5CE54087
:103FAA0075F00584ADF07C008D5F7564057532058A
:103FBA00753360E55CC3941750051230AD800690E6
:103FCA0005E6E0F55CE567255CC39464F567E5669C
:103FDA002567F55990007DE0B402109007B3E025FB
:103FEA0059FE9000D1E0F4042EF5599000D4E0D3A4
:103FFA0094014040E543C394E7501D74E7C39543D9
:10400A00FE9007B5E08E00F5F0E884FF7E008F5C35
:10401A00E559255CF559801CE543C394E7FE9007F2
:10402A00B5E08E00F5F0E884FF7E008F5CE559C3A9
:10403A00955CF559A2084006E5662464F559E559E8
:10404A00D394644009E559C39464F55980037559BA
:10405A00009000ADE0C3955950069000ADE0F559C7
:10406A0022D2009000C3E0A824B800049525503B52
:10407A009000C3E0A824B800049525500375590F91
:10408A009000C3E004A824B800049525500375598C
:10409A000A9000C3E02402A824B80004952550051C
:1040AA00755905C2007409900044F07E017F0090A2
:1040BA0000B3E0124AF19000C2E08E048F05FF12AD
:1040CA000085E537BC000CD39D4008C200740A90F5
:1040DA000044F09000B4E0C3953F500D9000C6E054
:1040EA00A824B80006952540028008C200740B90E7
:1040FA000044F0A200400375590590007DE0B40326
:10410A0006A201B3B34002802B900069E0C3940574
:10411A00A824B800049525500C90009EE0F5597427
:10412A000C900044F0900069E0A824B8000495259A
:10413A005002C20085594490006FE02559FE900054
:10414A0041E075F01E84FC7F00EE2CF559229000A8
:10415A0041E075F00584FF7E008F5C900041E075B8
:10416A00F00584ADF07C008D5F75640575320375CA
:10417A0033D69000C0E01475F00584FF7E00E55C3C
:10418A00BE00039F50051230AD800BE55C900445DC
:10419A00124B2DE0F55CE55C9007B6F09007B6E0AF
:1041AA00FE9000AFE0C39E50089000AFE09007B6C3
:1041BA00F022E53F75F00584FF7E0090056F124BF3
:1041CA0018E0F56BE56BD394644010E56BC3946417
:1041DA0075F00F84FF7E008F6B8003756B00900073
:1041EA0092E0256BF56B229007A9E0FEA3E0FF742D
:1041FA0004124AE3E537124AF1740F8E048F05FF61
:10420A001200859007A7ECF0A3EDF0900085E0B4CA
:10421A000262E542C3944175F00584FF7E008F5C1B
:10422A00E54275F00584ADF07C008D5F7564057517
:10423A003206753314E55CC3941750051230AD800D
:10424A0006900696E0F55C9007A7E0FEA3E0FF74EF
:10425A000A8E048F05FF120085E55C8C068D071215
:10426A004AF1740A8E048F05FF1200859007A7ECA5
:10427A00F0A3EDF09007A7E0FEA3E0FF9007ADE002
:10428A00FCA3E0FDEDD39FEC9E400F9007ADE0F854
:10429A00A3E09007A7C8F0A3C8F02290008CE0B46E
:1042AA00010385254F90008CE0B402129000C2E011
:1042BA008537F0A4FFAEF07408124AE38F4F9000DE
:1042CA008CE0B4030385394F90008CE0B404038575
:1042DA003F4F90008CE0B40507E540C39414F54FB6
:1042EA0090008CE0B4060385414F90008CE0B4073F
:1042FA000385424F90008CE0B4080385434F900039
:10430A008CE0B40903853E4F90008DE0FE90008E4C
:10431A00E0D39E404B90008CE0B4041890008EE0ED
:10432A00C3954F5002D20490008DE0D3954F4002BE
:10433A00C204802A90008DE0C3954F500990008EE8
:10434A00E0D3954F50028002D20490008DE0D395BD
:10435A004F500990008EE0C3954F5002C204802A44
:10436A0090008DE0D3954F400990008EE0C3954FA1
:10437A0040028002C20490008DE0C3954F4009902C
:10438A00008EE0D3954F4002D2042290008FE0B411
:10439A00010385254F90008FE0B402129000C2E01D
:1043AA008537F0A4FFAEF07408124AE38F4F9000ED
:1043BA008FE0B4030385394F90008FE0B40403857E
:1043CA003F4F90008FE0B40507E540C39414F54FC2
:1043DA0090008FE0B4060385414F90008FE0B40748
:1043EA000385424F90008FE0B4080385434F900045
:1043FA008FE0B40903853E4F900090E0FE90009153
:10440A00E0D39E4040900090E0C3954F5009900041
:10441A0091E0D3954F50028002D206900090E0D3EB
:10442A00954F5009900091E0C3954F5002C20690F3
:10443A00008FE0B401099000CEE0D3953950028094
:10444A0002C206802A900090E0D3954F400990005E
:10445A0091E0C3954F40028002C206900090E0C3EB
:10446A00954F4009900091E0D3954F4002D2062221
:10447A00AE57AF5874F5D39F74019E40087857120F
:10448A004B58024575755801755700AE24AF25E59E
:10449A006BBE000DD39F40099000A4E0D3956C40F9
:1044AA0002801B756C00E56BC39525F54F9000A73C
:1044BA00E0D3956A4006E56A254FF56A8002056CE5
:1044CA00900080E0D39539401CE537C395384015F4
:1044DA00AE24AF25E56BBE00039F50099000A5E00E
:1044EA00D3956D400280579007B7E0A824B800041E
:1044FA0095255003756F009007B7E0A824B8000B04
:10450A00D395254006E5259007B7F0E56F702AE5B3
:10451A0025C3956BF54FE54FD394054003754F05B9
:10452A009000A6E0C3956A5007E54FC3956A40021A
:10453A008007E56AC3954FF56A756D008002056DBF
:10454A00E56F7016900080E0C39539500DE56B2435
:10455A0005A824B8000695254002800F900093E034
:10456A00F56A756F0174789007B7F022AE57AF58A5
:10457A0074E9D39F74039E40087857124B58024738
:10458A0023755801755700756A32A21B402A756A4D
:10459A0019900093E075F002A4FFAEF0E56CBE003E
:1045AA0006D39F4002D21B056C756F03747890077F
:1045BA00B7F0756E00024712AE24AF25E56B6F4E59
:1045CA007003024712E56BBE000DD39F40099000AD
:1045DA00A4E0D3956C40028017756C00A208B3B3AF
:1045EA005007E56FC3940340028003756A19800D72
:1045FA00E56BC39525F54FE56C254FF56C9000806A
:10460A00E0D39539400E9007B7E0A824B80007D345
:10461A0095254002800C056E900093E0B56E0375F7
:10462A006F00E56FB4030DE56B2402A824B80006F9
:10463A0095254002800A056EE56EB43C03756F024B
:10464A00E56FB402299007B7E0A824B8000ED39505
:10465A00254009E5259007B7F0756E00900080E0C7
:10466A00C395395009756E0074789007B7F0E56FF5
:10467A00705A900080E0D39539401CE537D39538BD
:10468A004015AE24AF25E56BBE00039F500990008C
:10469A00A5E0D3956D40028008756D00756A4B8060
:1046AA0028E525C3956BF54FE54FD394054003756F
:1046BA004F05900080E0D395394008E56D254FF508
:1046CA006D8006E56D2406F56D756E00E56F701652
:1046DA00900080E0C39539500DE56B2405A824B8F5
:1046EA000006952540028003756F01E56FB4011835
:1046FA00756A19056E900093E0B56E06756F0275BE
:10470A006E0074789007B7F0E56A75F00AA4FFAEF8
:0A471A00F09007B1EEF0A3EFF022DB
:094B2D002582F582500205832265
:0F4AD40025E050020583258250020583F58222DA
:10006400EF2F500205832582F582E5833E2EF5832A
:010074002269
:104B4800CFC39FFF50011E22C3EF9DFFEE9CFE22A4
:094B3600E493F608740193F622E1
:084B58000806B600021806224F
:0D4AFF00A3E004F07006124B23E004F02247
:0E003900A3E014F0B4FF06124B23E014F022F3
:0E4AE300048007C3CE13CECF13CFD5E0F6224A
:1049F300BC000FBE0008ED8FF084FFADF022E4FE93
:104A0300FF22BE000DEF60FE54F0606F20E703024B
:104A13004AA9EAC0E0EBC0E078017A0075F001EE44
:104A230020E710EF25E0FFEE33FE0AC5F023C5F0C3
:104A330030E7F0EA5407F9096A7A007B006001085D
:104A4300C3EC9E40167004ED9F4010ED9FFDEC9E5D
:104A5300FCE5F0CA4ACA03F5F08005E5F003F5F07A
:104A6300C3EE13FEEF13FFD9D77908CACBCAD8D048
:104A7300EAFEEBFFD0E0FBD0E0FA22EC8FF084FCFF
:104A8300ED54F045F0C48FF084FEEDC454F045F0CE
:104A9300C48FF084FDEEC4FE54F02DFFEE540F3CA2
:104AA300FEADF07C0022790078008FF0EC7E0820C8
:104AB300E70DC3CD33CD33C933C9C833C8DEF08462
:104AC30049F9E5F08FF0BE00E6FD7C00E9FFE8FE62
:014AD30022C0
:0E4AF100F88FF0A4FFE5F0CE88F0A42EFE2290
:10000300EF8DF0A4F9A8F0EF8CF0A428F8EE8DF0B2
:06001300A428FEE9FF2213
:10007500600D782B02007F007830D8FED5E0F8229D
:10008500EEC0E07E001249F3EFFDEEFCD0E0FE226B
:0C4B0C00EEC0E07E001249F3D0E0FE2273
:03001B0002001EC2
:03009B0002004917
:03000000024B3F71
:094B3F0075817075D00002049E1E
:104B1800E5822FF582E5833EF583220582D5820260
:054B2800158315822237
:10001E00C0E0C0F0C083C082C0D075D000120455BD
:0B002E00D0D0D082D083D0F0D0E032E0
:10004900C0E0C0F0C083C082C0D075D0001204588F
:0B005900D0D0D082D083D0F0D0E032B5
:00000001FF
